:100000000C942A000C9447000C9447000C94470071
:100010000C9447000C9447000C9447000C94470044
:100020000C9447000C9447000C9447000C94470034
:100030000C9447000C9447000C9447000C94470024
:100040000C9447000C9447000C9447000C94470014
:100050000C94470011241FBECFE5D4E0DEBFCDBF16
:1000600010E0A0E6B0E0EEE3F2E002C005900D92F1
:10007000A237B107D9F710E0A2E7B0E001C01D92A6
:10008000A237B107E1F70E948C000C941E010C947A
:100090000000AC01892B59F020E030E08AEF90E0BD
:1000A0000197F1F72F5F3F4F24173507B9F70895F0
:1000B000BB9ABC98BD9A8A98BA9AA19AA39A0895B5
:1000C000C29AC39AC59880B386B3A99A0895C59871
:1000D000C29820E0C598C598992314F4C39A01C02A
:1000E000C398C59AC59A2F5F203119F0880F991FC0
:1000F000F1CFC598C29A089590E08299FECF829B75
:10010000FECF882314F4A99A01C0A9989F5F983064
:1001100010F4880FF2CF0895CF92DF92EF92FF9202
:100120000F931F93CF93DF930E9458000E946000AB
:10013000AB9A84E690E00E94490080E09CEC0E942B
:10014000670082E790E90E94670080E496EA0E94D7
:10015000670080E490ED0E94670081E198EC0E94C6
:10016000670080E292EC0E94670081E090EC0E94C0
:10017000670080E090EB0E94670000E00F2EF0E641
:10018000CF2EF0E0DF2EF02DEE24FF246894E4F86B
:10019000EC0CFD1CAB9A89E390EC0E94670010E028
:1001A0008AEA0E947C001F5F1330D1F78DE20E9423
:1001B0007C0084ED0E947C00E60110E088810E94B2
:1001C0007C008991180FCE15DF05C1F7812F0E94A1
:1001D0007C008AEA0E947C008AEA0E947C0081E01E
:1001E00090EC0E946700AB9884EF91E00E94490078
:1001F0000F5F802F64E60E941201805D80936D0086
:10020000802F0E941201292F892F6AE00E9412017B
:10021000805D80936E00822F0E941201905D90930A
:100220006F00B8CF991B79E004C0991F961708F0AA
:0E023000961B881F7A95C9F780950895FFCF19
:10023E000A0D41546D65676131360A0D202D2D2D45
:02024E000000AE
:00000001FF
